:020000040801F1
:10C0000000C0002085D7010801D9010855DA0108D0
:10C0100065DA010869DA01086DDA0108000000003C
:10C020000000000000000000000000000000000010
:10C030000000000000000000000000000000000000
:10C0400000000000000000000000000000000000F0
:10C0500000000000000000000000000000000000E0
:10C0600000000000000000000000000000000000D0
:10C0700000000000000000000000000000000000C0
:10C0800000000000000000000000000071DA01085C
:10C0900075DA010800000000000000000000000048
:10C0A0000000000000000000000000000000000090
:10C0B0000000000079DA0108000000000000000024
:10C0C0000000000000000000000000000000000070
:10C0D0000000000000000000000000000000000060
:10C0E0000000000000000000000000000000000050
:10C0F0000000000000000000000000000000000040
:10C10000000000000000000000000000000000002F
:10C11000000000000000000000000000000000001F
:10C12000000000000000000000000000000000000F
:10C130002DE9F047884282B00F46144653D2061DBF
:10C140004FF664688E1B0546C0F6010802E0043E07
:10C15000AF4248D955F8049B5FFA89F000F044FDDE
:10C1600021885FFA89F0CB0303EB510C0CEB000242
:10C170004FEA192A5FFA8AF0228000F035FD218803
:10C180005FFA8AF0CB0303EB510C0CEB00024FEA91
:10C19000194A5FFA8AF0228000F026FD23885FFAB0
:10C1A0008AF0D90301EB530A82444FEA19694846E1
:10C1B000A4F800A000F018FD21886805CA0302EB6E
:10C1C00051039944400DA4F800900028BFD10146C6
:10C1D0004FF6FF7203460196CDF80080043E00F052
:10C1E000A1FAAF42B6D802B0BDE8F08730B5002062
:10C1F0004FF68C6585B001464FF6FF720346C0F6D8
:10C20000010504AC009500F08DFA00234FF6A06004
:10C2100024F8023DC0F6010000F0C8FC00212246CF
:10C22000C0F604014FF00060FFF782FF4FF6AC64E8
:10C2300000F008FD0020BDF80E50C0F601040146D4
:10C240004FF6FF7203468DE8300000F06BFAFEE710
:10C25000CB7970B49842CE682AD3012203FB02F254
:10C26000B0FBF2F49C42F9D2E2B1002502FB1400CB
:10C27000B2FBF3F20DB9002C0FDD092C16DD0B7AA1
:10C28000002B0CBF572337231C1906F8014B4AB16A
:10C29000CB790135B0FBF2F4E8E7002AFAD130346B
:10C2A00006F8014B0020307070BC70473023EBE77C
:10C2B00001220446D9E700BF2DE9F843D3681746A9
:10C2C0001A7805460E463C68A2B1002C12DD13F820
:10C2D000010F013C04F0010160B15CB109B104E05F
:10C2E00044B113F8011F013C21B113F8012F013CA7
:10C2F000002AF5D1797901B1013CBB792BB1FB79E9
:10C30000102B61D0082B08BF013C387910BB631E8D
:10C31000002C6CDD20214FF00108284603EA0809B3
:10C32000B047A04513D0B9F1000F06D02021284610
:10C330004FF00208B047A04509D020212846B04759
:10C3400008F1020820212846B047A045F5D17979A7
:10C350004FF0FF34002934D1B97921B1FB79102B8A
:10C3600034D0082B3FD03A7902B3002C1EDD3021A7
:10C370004FF00108284604F1FF39B047A04509EA0B
:10C38000080913D0B9F1000F06D0302128464FF02C
:10C390000208B047A04509D030212846B04708F12F
:10C3A000020830212846B047A045F5D1FC68217825
:10C3B00029B12846B04714F8011F0029F9D1BDE87A
:10C3C000F8832846B047C7E7023C9EE7284630215D
:10C3D000B04797F808C02846BCF1000F0CBF782181
:10C3E0005821B047BFE728463021B047BBE71C467D
:10C3F000B0E700BF436882680133934205D2026808
:10C40000436002F8011B026070474360704700BF41
:10C410002DE9F04188B0984605AB06460D46144616
:10C42000049300272178002942D0013425293AD1EC
:10C4300001978DF8097038463B4614F8011B002916
:10C4400036D0232963D030295FD0A1F130025FFAC2
:10C4500082FCBCF1090F8DF808008DF80A3012D863
:10C460000023D0B2A1F1610C09285FFA8CFC22D91B
:10C47000A1F14102BCF1050FD2B225D8A1F15702BA
:10C480000A2A18DD01936C2908BF14F8011B6929D9
:10C490004BD03ED8632969D044D858291DD0C1D883
:10C4A00031B12529BED13046A84721780029BCD119
:10C4B00008B0BDE8F08114F8011B03EB830002EB28
:10C4C0004003A1F13002CCE7052ADBD8A1F1370205
:10C4D000D6E775293BD07829A4D1A1F15801D1F133
:10C4E000000C4CEB010E10208DF80B008DF80CE0C9
:10C4F000D8F8000001A9FFF7ABFE3046294601AA93
:10C5000008F10408FFF7D8FE8CE7012095E7012326
:10C5100093E773291FD0DCD86F2983D108238DF8C6
:10C520000B30E5E764297FF47DAF0A238DF80B30EB
:10C53000D8F8000008F1040800281EDB01A9FFF765
:10C5400087FE3046294601AAFFF7B6FE6AE70A21B0
:10C550008DF80B10CCE7D8F800303046294601AAF8
:10C5600008F104080493FFF7A7FE5BE798F80010B2
:10C57000304608F10408A84754E72D22404201A99B
:10C580008DF80920FFF764FE3046294601AAFFF71F
:10C5900093FE47E710B584B001900024039101A8F1
:10C5A00004490294FFF734FF019B1C70029804B009
:10C5B00010BD00BFF5C301080CB410B582B004ACC7
:10C5C00054F8042B23460194FFF7E4FF02B0BDE8C2
:10C5D000104002B0704700BF70B40278002A47D004
:10C5E000254C0023E51D202107E090F800C004F849
:10C5F00003C010F8012F01331AB32E2AF5D10130F0
:10C60000072BF2DC5E1EA219D343EE18531CAB427B
:10C61000517006F001060AD01EB103F8011FAB42AB
:10C6200005D05A1C59700233AB425170F9D190F8C1
:10C6300000C0082304F803C010F8012F0133002ABA
:10C64000DBD10A2B11DC5A1C20210A2AE15403F009
:10C6500001030ADC1BB1A15401320A2A05DC501C7B
:10C66000A15402320A2A2154F9DD034870BC7047F4
:10C670001346014CE7E700BF043100209CF802306C
:10C680002DE9F0416446154613B1024608461146AD
:10C69000C1F30F21C0F30F20E7F7B8FDE7F7E4FD82
:10C6A000C5F580721E49550081FB05372388C7EB0D
:10C6B000E57C03F4FC640CF58075E61006FB05F6DA
:10C6C000DA0003F4784700F4FC613F1202F0FF0443
:10C6D000C5F5807CCA1004FB05F407FB05F50CFBCF
:10C6E000026200F47843C10018120CFB0050002ACB
:10C6F00001F0FF01B8BFFF320CFB014193125A0158
:10C700000028B8BFFF30C312002942EAC320B8BFD7
:10C71000FF3140EAE12188B2BDE8F041E7F778BD9A
:10C72000565555552DE9F04385B00DF1300E5EF8A4
:10C7300004CB0C4C06460F46154698466246734697
:10C7400037212046CDF80CE0FFF724FF394681461B
:10C750002A46304643460094E7F776FD484605B042
:10C76000BDE8F0831031002008B42DE9F04F88B007
:10C7700011AF57F8045B00F1100302970390029881
:10C780003E4F041D11958846924605934FF00009CF
:10C7900004944FF6487B0020394D4146024603463B
:10C7A0000095FFF7BFFF119C4146524600230398B6
:10C7B0000094E7F749FD119803F024FB029A0499CD
:10C7C00014680791002C57D0059E002506EBC00683
:10C7D000C9EB050EDEF1000C4CEB0E03B0B2414686
:10C7E00052460094E7F730FD204603F00BFB079913
:10C7F00002300C680B1D06EBC00601350793002CB8
:10C80000E6D164223A803B889CB2002CFBD1042004
:10C81000E7F720FD80F47E4C8CF4A47448F24801C4
:10C8200004EA01000028F2D00420E7F713FD584580
:10C83000FAD164223A80B7F800E01FFA8EF3002B99
:10C84000F9D114F0080F05D0B9F1000F02DD09F19C
:10C85000FF39A0E714F4004F05D0013DA94502DAE5
:10C8600009F1010997E714F0400F94D0484608B049
:10C87000BDE8F04F01B070472546C2E7987200202E
:10C880000CFF01082DE9F04F83B01446BDF83020AD
:10C8900088461E464FF087410023ADF804208DF8EE
:10C8A000063003F09DF803F061FA4FF08741074628
:10C8B000204603F095F803F059FA4FF087410446FB
:10C8C000404603F08DF803F051FA4FF0874181465E
:10C8D000304603F085F803F049FAE31BC9EB000288
:10C8E00083EAE375A5EBE37582EAE271A1EBE271FD
:10C8F0008D4280F2CB80BA4601279846A3468DF838
:10C900000670134604464F46BC4205DAD146384607
:10C91000DA462746CB46044607F1800C2CF0FF058B
:10C920004FEA0828EA1B98FBF3F808FB02F10029FC
:10C93000B8BFFF310AEB212A0CF0FF000AF0FF0715
:10C94000C7F5807EC0F5807606FB0EF306FB07F682
:10C950002AF0FF091A12284649460DF1040CFFF788
:10C960008DFE3212284609F580710DF1040CFFF797
:10C9700085FE04F1800222F0FF09C4EB090708FBE1
:10C9800007F4002CB8BFFF340BEB242C0CF0FF078E
:10C9900002F0FF06C7F5807106FB01F306FB07F600
:10C9A0002CF0FF041A120DF1040C48462146FFF743
:10C9B00065FE0135320A0DF1040C484604F580711C
:10C9C000FFF75CFE4D455EDA0AEB080626F0FF072E
:10C9D00006F0FF0AEC4328463946CAF580720DF18D
:10C9E000040CFFF74BFE04EB090B284605F5807499
:10C9F0000DF1040C07F580715246FFF73FFE4C45E0
:10CA0000CBF3002B06EB08053DDABBF1000F0AD093
:10CA100025F0FF0705F0FF0620463946C6F580726F
:10CA20000DF1040C20E025F0FF0705F0FF0620467D
:10CA30003946C6F5807245440DF1040CFFF71EFE21
:10CA4000204607F5807132460DF1040C04F5807420
:10CA500025F0FF0705F0FF06FFF710FE3946C6F583
:10CA600080720DF1040C2046FFF708FE20460DF100
:10CA7000040C07F58071324604F58074FFF7FEFD63
:10CA80004C454544CFDB03B0BDE8F08F904683466C
:10CA9000CA4639E788422DE9F04105460C461E4654
:10CAA0002DDC97B23946C0EB040880B2E7F7AEFB45
:10CAB00002353046E7F7ACFBAC42C8F3400820DB58
:10CAC000B8F1000F09D0A8B23946E7F79FFB02354D
:10CAD0003046E7F79DFBAC4215DB3946A8B2E7F7D5
:10CAE00095FB02353046E7F793FBA8B23946E7F7E6
:10CAF0008DFB02353046E7F78BFBAC42EDDABDE843
:10CB0000F081BDE8F081BDE8F08100BF91422DE9E0
:10CB1000F0410C4615461E462DDC87B289B23846D8
:10CB2000C4EB0208E7F772FB02343046E7F770FB0C
:10CB3000A542C8F3400820DBB8F1000F09D0A1B22C
:10CB40003846E7F763FB02343046E7F761FBA5425E
:10CB500015DBA1B23846E7F759FB02343046E7F758
:10CB600057FBA1B23846E7F751FB02343046E7F7EE
:10CB70004FFBA542EDDABDE8F081BDE8F081BDE8EC
:10CB8000F08100BF08B5FFF727FD074B014603F50D
:10CB9000277203F1440003F52973E7F777FBD0F11F
:10CBA000010038BF002008BD0431002010B5FFF798
:10CBB00013FD0C4C014604F5297304F1440004F5FF
:10CBC0002772E7F761FB0023C11A484240EB0100DE
:10CBD00084F8A802C4F8AC32C4F8B032C4F8B43255
:10CBE00010BD00BF0431002038B5144C94F8A832B1
:10CBF0007BB1D4F8B032D4F8AC22E1180133013261
:10CC0000B3F5007F81F84400C4F8B032C4F8AC2218
:10CC100000D238BDD4F8B4020025421C04F52771B7
:10CC200004F14400C4F8B052C4F8B422E7F732FB70
:10CC30000028EED084F8A85238BD00BF043100208F
:10CC40000846D1E738B5104C94F8A80218B919E095
:10CC50002020FFF7C9FFD4F8B032002BF8D10B48E1
:10CC6000D4F8B4120025490200F5167200F51873C5
:10CC700084F8A852E7F710FBC5EB000CDCF10000CC
:10CC800040EB0C0038BD00BF0431002048310020CB
:10CC90000FB470B582B006AE56F8042B084C0020D5
:10CCA00008493346D4F8AC520196FFF7B1FBD4F8EB
:10CCB000AC02401B02B0BDE8704004B0704700BF3A
:10CCC0000431002041CC010870B50646002409E07B
:10CCD0000D48FFF771FC0C48FFF754FF90B1B4F515
:10CCE0007A7F0FD023460D2132460748FFF764FCB8
:10CCF0000548FFF747FF651C0D21023432462B46DD
:10CD00000028E5D1004870BDBC3300202DE9F00FAC
:10CD1000C20000F4FC64E41002F0FF0200F4784169
:10CD20000912A4F1FC05A2F1F80685EAE579A9EB60
:10CD3000E57986EAE678A8EBE678A1F1F80C8CEACA
:10CD4000EC77A7EBEC77A01809EB08034018DB1988
:10CD5000984200F3DA8003460020A4F1800BA2F190
:10CD60008008A1F1800788EAE879A9EBE8798BEAE5
:10CD7000EB7AAAEBEB7ACA4487EAE779A9EBE77981
:10CD8000D1444B45C4BF4B46022086EAE67AAAEB63
:10CD9000E67A04EB0A0909EB010A5345C4BF53467E
:10CDA000032085EAE579A9EBE57909EB020A0AEBAC
:10CDB00001094B45C8BF4B4604EB020AC8BF04201B
:10CDC0008CEAEC79A9EBEC79D1444B45C4BF4B46D6
:10CDD000052086EAE679A9EBE67985EAE57AAAEB09
:10CDE000E57ACA440AEB01094B45C4BF4B4606200D
:10CDF00085EAE57AAAEBE57A92448CEAEC79A9EB2C
:10CE0000EC79D1444B45C4BF4B46072086EAE6790E
:10CE1000A9EBE679BCF1000FB8BFCCF1000CA1443E
:10CE2000E1444B45C4BF4B46082088EAE87CACEBA4
:10CE3000E87C04EB0C0909EB010C6345C4BF6346B5
:10CE400009208BEAEB79A9EBEB7909EB020C0CEBEF
:10CE500001094B45C4BF4B460A2004EB020987EA8F
:10CE6000E77CACEBE77CCC446345C4BF63460B2056
:10CE700085EAE57CACEBE57CB8F1000FB8BFC8F102
:10CE80000008E04487EAE77CACEBE77CC4446345F8
:10CE9000C4BF63460C20002EB8BF7642002DB8BF39
:10CEA0006D42AD19002FB8BF7F42EF19BB42C8BF1A
:10CEB0003B46A2F1600CC8BF0D20BC3C84EAE4767E
:10CEC000A6EBE476BCF1000FB8BFCCF1000C6039E2
:10CED000664481EAE175A5EBE1757519AB42C4BF03
:10CEE0002B460E20B83A002CB8BF6442002AB8BFC7
:10CEF0005242A4180029B8BF494204EB010C9C45DA
:10CF0000B8BF0F20BDE8F00F7047012025E700BF34
:10CF10002DE9F041FFF74AFE874C04F136066078B0
:10CF2000651CFFF761FE02346878FFF75DFEB442CE
:10CF3000F5D10020FFF758FE0020FFF755FE002036
:10CF4000FFF752FE0020FFF74FFEF820FFF74CFEE0
:10CF5000FC20FFF749FEF820FFF746FE0020FFF710
:10CF600043FE8020FFF740FE8020FFF73DFE80203B
:10CF7000FFF73AFE0020FFF737FE0020FFF734FEF0
:10CF80000020FFF731FEF820FFF72EFE0020FFF70C
:10CF90002BFE0020FFF728FEFC20FFF725FE0020D7
:10CFA000FFF722FE0020FFF71FFEF820FFF71CFE10
:10CFB0000020FFF719FE0020FFF716FE0020FFF704
:10CFC00013FE0020FFF710FEFC20FFF70DFEF820F7
:10CFD000FFF70AFE0020FFF707FEF820FFF704FE28
:10CFE000FC20FFF701FE0020FFF7FEFD0020FFF709
:10CFF000FBFDF820FFF7F8FD0020FFF7F5FDF82016
:10D00000FFF7F2FD0020FFF7EFFD0020FFF7ECFD3A
:10D010000020FFF7E9FD8020FFF7E6FD0020FFF785
:10D02000E3FD0020FFF7E0FD8020FFF7DDFD00209D
:10D03000FFF7DAFD0020FFF7D7FD8020FFF7D4FDD2
:10D040000020FFF7D1FD0020FFF7CEFD0020FFF705
:10D05000CBFD8020FFF7C8FDFC20FFF7C5FD802039
:10D06000FFF7C2FD0020FFF7BFFD8020FFF7BCFDEA
:10D07000FC20FFF7B9FDF820FFF7B6FD0020FFF711
:10D08000B3FD6020FFF7B0FDBC20FFF7ADFD6020D1
:10D09000FFF7AAFD0020FFF7A7FD6020FFF7A4FD22
:10D0A000BC20FFF7A1FDB820FFF79EFD0020FFF791
:10D0B0009BFD4FF0000840F291171FFA88F50124FC
:10D0C000601E294680B2E7F7A1F8E7F7CDF8FFF731
:10D0D0001DFE294606462046E7F798F8E7F7C4F80C
:10D0E000FFF714FE40EA0613D8B2FFF77DFDA11C3E
:10D0F0008CB2621E90B22946E7F788F8E7F7B4F8D9
:10D10000FFF704FE294606462046E7F77FF8E7F7D3
:10D11000ABF8FFF7FBFD023440EA0610C0B2A4B240
:10D12000FFF762FDBC42CBD108F10108B8F1F00F66
:10D13000C3D1BDE8F04185E5D3FE0108034B18805B
:10D14000188882B2002AFBD1704700BF9872002075
:10D150002DE9F04F40F66A78044608FB00F00028FD
:10D16000B8BF033087B07A4E04928210B6FBF2F655
:10D17000784D0293731C95FBF3F5059140F66A77A1
:10D1800095FBF4F197FBF1F005FB00F2202092FBF8
:10D19000F4F301460193E7F759F807200021E7F778
:10D1A00055F808203146E7F751F800208021E7F7CD
:10D1B0004DF8694A51680129FCD1674A5768012F27
:10D1C000FCD006200121E7F741F80320E7F742F8F9
:10D1D0000028FAD000260236E7F72CF8E7F72AF8FD
:10D1E000962EF8D1204602F0A7FB5C4902F0F8FB2E
:10D1F0008146284602F0A0FB0146484602F0A4FC06
:10D20000019C0390002C40F3988000260024B14636
:10D21000A046FF272EE002F08FFB0546204602F0D5
:10D220008BFB039902F0DCFB824600F0B1FC8346E5
:10D23000504600F0E3FC0021824602F0D1FB01469B
:10D24000584602F0C3FA0146284602F0C9FB0146DF
:10D25000484602F0BDFA0AF100418146284602F034
:10D26000BFFB0146304602F0B3FA019A0134944202
:10D27000064614D0E6F7DEFF029D5FFA80FC6046AA
:10D28000E045B8BFE0466745A8BF6746002DC2D15C
:10D29000049B002BBFD1019A01349442EAD1019B37
:10D2A000059C03EBD370C7EB08072760401002F022
:10D2B00043FB05462946484602F046FC29460446FB
:10D2C000304602F041FC21460546204602F088FB2C
:10D2D00029460646284602F083FB0146304602F006
:10D2E00077FA00F0C9FC0499064621B11C4902F006
:10D2F0002BFC049A1060029941B130464FF08041F6
:10D3000002F02AFD28B9174B0298036007B0BDE868
:10D31000F08F05F10041204600F0ACFC124902F00C
:10D320005FFB01F099FF08A3D3E9002302F012F993
:10D3300002F0F8F9029B1860E8E700264FF00008B9
:10D34000B146FF27ABE700BF182D4454FB2109402D
:10D35000FFA14A0400A24A0444040240DB0FC94072
:10D36000F304B53F0000C07F0000344310B5002136
:10D3700082B004460A20E6F769FF0220FFF7DEFECE
:10D3800000221346204601A9FFF7E2FE019BC72BAE
:10D3900073DD01210A20E6F759FF0220FFF7CEFED8
:10D3A0000022204601A91346FFF7D2FE0198C728A4
:10D3B00065DD02210A20E6F749FF0220FFF7BEFEE5
:10D3C000002201A920461346FFF7C2FE0199C72992
:10D3D00057DD03210A20E6F739FF0220FFF7AEFEF2
:10D3E00000221346204601A9FFF7B2FE019AC72A80
:10D3F00049DD04210A20E6F729FF0220FFF79EFEFF
:10D4000000221346204601A9FFF7A2FE019BC72B6D
:10D410003BDD05210A20E6F719FF0220FFF78EFE0B
:10D420000022204601A91346FFF792FE0198C72863
:10D430002DDD06210A20E6F709FF0220FFF77EFE18
:10D44000002201A920461346FFF782FE0199C72951
:10D450001FDD07210A20E6F7F9FE0220FFF76EFE26
:10D4600000222046134601A9FFF772FE019AC72A3F
:10D47000CCBF0820072002B010BD0020FBE7012030
:10D48000F9E70220F7E70320F5E70420F3E705209A
:10D49000F1E70620EFE700BF70B50C4682B02346E7
:10D4A00001A96A460646FFF753FE019B143BD22BA7
:10D4B00013D8104D0720E6F7CDFE2A6802EB820153
:10D4C00000EB8100006902F037FA009902F088FA57
:10D4D000094902F039FB02B070BD3046FFF746FF44
:10D4E000044D01A928606A4630462346FFF730FE06
:10D4F000E0E700BF0030002000247449AFF3008053
:10D500002DE9F04104461046884602F015FA3749E5
:10D5100002F066FA0546404602F00EFA0146284639
:10D5200002F012FBB8F1000F07465CDD0020002678
:10D5300018F0010F05463AD12D4902F051FA2C4955
:10D5400002F046F902F038FC394624F8020B28466E
:10D5500002F03EF92549054602F0FEFB20B12846BF
:10D56000224902F033F90546284600F047FB012620
:10D570001DE000F043FB1E4902F032FA1C4902F0A4
:10D5800027F902F019FC394624F8020B284602F06C
:10D590001FF91649054602F0DFFB144918B1284669
:10D5A00002F014F90546284600F028FB0136104920
:10D5B00002F016FA0E4902F00BF902F0FDFB3946B3
:10D5C00024F8020B284602F003F90849054602F048
:10D5D000C3FB0136054918B1284602F0F7F80546A5
:10D5E00046452846C5D1BDE8F08100BFDB0FC940E4
:10D5F00000E0FF444FF4FA5C2DE9F0410CFB00F42D
:10D600002249651EA1FB0516B20C0132204BB4FB6A
:10D61000F2F7B3FBF7F74FF6FF784745A8BF474649
:10D620001C4D791C95FBF1F602FB06F606EB500447
:10D63000DFF86C80184BB4FBF0F44FF0000EB4F53B
:10D64000FA5FA8BF4FF4FA54144DA3F828E04046FF
:10D650002146FFF755FF2B680F2023F001022A60B7
:10D660002146E6F7F3FD0E204146E6F7EFFD296877
:10D670000D2041F001032B603946E6F7E7FD06EB8C
:10D680005400B0FBF4F0BDE8F08100BF83DE1B4323
:10D69000FFA14A0400A24A040014004044040240CE
:10D6A000CC33002010B50D4C0021B4FBF0F4621C0B
:10D6B00012F0010F08BF14461020E6F7C7FD112035
:10D6C000611EE6F7C3FD12206108E6F7BFFD0449BD
:10D6D00063085818B0FBF4F010BD00BFFFA14A0466
:10D6E00000A24A042248234970B4884223D0224C25
:10D6F000A14220D2024652F8046B0B46CD4343F8B8
:10D70000046B6519A342C5F3800514D23DB11568B9
:10D7100000F108021D6001F10803A3420BD210467C
:10D7200050F8045B194641F8045B5568021D5D60C2
:10D730000B1DA342F3D3114A1148824216D2002195
:10D740001346D44343F8041B04198342C4F38004F2
:10D750000CD224B1196002F10803834206D21A46A2
:10D7600042F8041B5960131D8342F8D370BC704704
:10D77000F4030208003000200431002004310020AE
:10D78000B4720020054B064ADFF818D09A60FFF704
:10D79000A9FFE6F76BFDFEF729FDFEE700ED00E0CF
:10D7A00000C0010800C00020F0B50A2883B009D0ED
:10D7B0000E4C27683F2F07D0E11901370871276009
:10D7C00003B0F0BD094C2768094D0026E7193E71EA
:10D7D000084F334629880A204FF6FF720097E6F774
:10D7E00033FD2B6826600E3B2B60E9E74C7200206E
:10D7F000043000205072002010B50446007828B193
:10D80000FFF7D2FF14F8010F0028F9D110BD00BFB7
:10D8100010B50446C0780009092839DD3730FFF714
:10D82000C3FFE17801F00F00092839DD3730FFF739
:10D83000BBFFA2781009092839DD3730FFF7B4FFA4
:10D84000A37803F00F00092839DD3730FFF7ACFF6C
:10D8500060780009092839DD3730FFF7A5FF94F813
:10D8600001C00CF00F00092839DD3730FFF79CFFAD
:10D8700021780809092839DC3030FFF795FF227834
:10D8800002F00F00092839DC3030BDE810408BE78A
:10D890003030FFF789FFE17801F00F000928C5DC7F
:10D8A0003030FFF781FFA27810090928C5DC30303D
:10D8B000FFF77AFFA37803F00F000928C5DC3030AA
:10D8C000FFF772FF607800090928C5DC3030FFF7E8
:10D8D0006BFF94F801C00CF00F000928C5DC303054
:10D8E000FFF762FF217808090928C5DD3730FFF707
:10D8F0005BFF227802F00F000928C5DD3730C4E74E
:10D90000704700BF002038B50146E6F77FFC3F486E
:10D910004BF68031E6F788FC3C484BF68031E6F761
:10D9200083FC00210320E6F791FC394C3948FFF7CE
:10D9300063FF3948FFF760FF04F14400FFF768FF19
:10D940003648FFF759FF606C00251830FFF760FF7D
:10D950003348FFF751FF606C1430FFF759FF31482F
:10D96000FFF74AFF606CFFF753FF2F48FFF744FFB4
:10D97000606C0430FFF74CFF2C48FFF73DFF606CF4
:10D980000830FFF745FF2A48FFF736FF606C0C3080
:10D99000FFF73EFF2748FFF72FFF606C1030FFF7BF
:10D9A00037FF2548FFF728FF2448FFF731FF2448B9
:10D9B000FFF722FF2348FFF72BFF2348FFF71CFF49
:10D9C00005E02248FFF718FF0135202D1AD0606CC2
:10D9D00000EB8500FFF71CFF05F00302032A1B483C
:10D9E00008BF1B48FFF708FF616C013501EB85009C
:10D9F000FFF70EFF05F00303032BE2D11448FFF7F6
:10DA0000FBFEE1E71248FFF7F7FEFEE708300020D3
:10DA10004C72002054FF010884FF01088CFF0108AC
:10DA200094FF01089CFF0108A8FF0108B0FF01084E
:10DA3000BCFF0108C4FF0108CCFF01082CED00E089
:10DA4000D8FF010828ED00E0E4FF010880FF01088D
:10DA5000F0FF0108024BEFF308825A6452E700BF5F
:10DA60004C720020FEE700BFFEE700BFFEE700BFEC
:10DA7000E6F7C6BBE6F7C6BB38B5444C1320A36C2B
:10DA800000215A1CA264E6F7E1FBB4F84C0083B213
:10DA900023B1B4F84C00411EA4F84C1094F84E2069
:10DAA0003A4B002A4BD1142283F84E201D6D15B13C
:10DAB000186D411E1965B4F854E0344B1FFA8EFC02
:10DAC000BCF1130F41D9B3F85450143DA3F854508E
:10DAD00094F856302D4D312B40D895F856104A1CED
:10DAE00085F8562094F85C10284B4A1C84F85C207A
:10DAF00094F85CE0BEF10B0F0ED9002283F85C2095
:10DB000093F85DE0DEF1010C38BF4FF0000C01200E
:10DB100083F85DC083F85E0094F85F101B4B21B161
:10DB200093F85F20501E83F85F0094F86010174B45
:10DB300021B193F86020501E83F8600038BD93F83F
:10DB40004E00411E83F84E1038BD03200021E6F739
:10DB50007DFB94F856300D4D312BBED900230420A7
:10DB600085F856300121E6F771FBB5F85820531CB3
:10DB7000A5F85830B5F85AC01FFA8CF00028B1D07B
:10DB8000B5F85A00411EA5F85A10ABE74C720020B8
:10DB900040F6D87320F00042C3F6497301469A421A
:10DBA00000B583B015DDB2F1FF4F03DB01F00EFECF
:10DBB00003B000BD694600F05DF900F00302009873
:10DBC000012A10D0022A08D09AB9019900F056FB18
:10DBD000EEE7002100F052FBEAE7019900F04EFB6E
:10DBE00000F10040E4E7019900F03AFF00F1004045
:10DBF000DEE70122019900F033FFD9E740F6D87340
:10DC000020F00042C3F6497301469A4200B583B042
:10DC100016DDB2F1FF4F03DB01F0D8FD03B000BD0C
:10DC2000694600F027F900F00300012815D002280A
:10DC30000BD0B8B900980122019900F011FFEDE76F
:10DC40000021002200F00CFFE8E700980122019972
:10DC500000F006FF00F10040E0E70098019900F0B5
:10DC60000DFBDBE70098019900F008FB00F1004094
:10DC7000D4E700BF00F052B870B58AB0064600F095
:10DC8000A5FA43F20C04C2F2000494F90030013307
:10DC9000054630D0304601F0D5F800282BD030466C
:10DCA000002102F03BF830B34FF6F4733046C0F673
:10DCB00001030193012300930023089301F0CCFAA0
:10DCC0002478CDE90401CDE90201BCB10020002196
:10DCD00002460B4601F03EFC022CCDE9060111D1B3
:10DCE00002F08AF821230360089B8BB9DDE9060165
:10DCF00001F018FD054628460AB070BD0022002339
:10DD0000CDE90623684600F02BFF0028ECD1E7E7B9
:10DD100002F072F8089B0360E8E700BFF8B520F056
:10DD20000044B4F1FF4F21F00046D4BF0027012783
:10DD3000B6F1FF4FC8BF47F001070346002F45D19A
:10DD4000B1F17E5F4CD08F1707F0020747EAD0771A
:10DD50004CB9022F3FD0032F03D140F6DB73CCF236
:10DD600049031846F8BD36B3B6F1FF4F55D0B4F1AC
:10DD7000FF4F20D0A41BE4153C2CC4BF40F6DB7041
:10DD8000C3F6C97030DD012F08BF00F10043E8D0B1
:10DD9000022F33D00346002FE3D04BF62E51C3F2AF
:10DDA000BB3101F015FD40F6DB71C4F2490101F011
:10DDB0000DFD0346D5E7002840F6DB73B8BFCBF670
:10DDC000C973CEDBC3F6C9731846F8BD01F000FD78
:10DDD00003461846F8BD40F6DB73C4F24903C0E7BA
:10DDE000BDE8F84000F0BEBE14F13C0FACBF00240B
:10DDF000012414EAD1741DD00020C4E74BF62E5143
:10DE0000C3F2BB3101F0E4FC014640F6DB70C4F222
:10DE1000490001F0DBFC0346A3E7B4F1FF4F10D04B
:10DE2000022FD8D0032F98D00023012F99D14FF083
:10DE3000004396E701F088FE00F0B2FF00F092FE8A
:10DE4000A1E7022F04BF4CF6E433C4F2160388D0D6
:10DE5000032F04BF4CF6E433CCF2160381D0012F1C
:10DE600040F6DB7318BFC3F649737FF47AAFCBF685
:10DE7000497376E740F6D8732DE9F04FC3F649733E
:10DE800020F0004B89B09B4505460C4640F38C8042
:10DE90004CF6E333C4F216039B4526DC00284FF40E
:10DEA0007861C3F6C97140F3538101F08FFC4FF4E0
:10DEB0007D632BF00F0BC3F6C9739B45054600F03D
:10DEC000828044F243410126C3F2357101F07EFCA9
:10DED00001462060284601F079FC44F24341C3F238
:10DEE000357101F073FC606062E04FF47863C4F256
:10DEF00049339B4540F38280BBF1FF4F5CDA4FEA28
:10DF0000EB59A9F186094FEAC953C3EB0B0B5846ED
:10DF100001F02CFF01F010FD034601465846059321
:10DF200001F054FC4FF0874101F05AFD064601F024
:10DF30001DFF01F001FD014607463046069701F03E
:10DF400045FC4FF0874101F04BFD0021032607906F
:10DF500001F0DAFE88B10326384600210DF11808D9
:10DF6000013E01F0D1FE40B158F8047D0021013E90
:10DF7000384601F0C9FE0028F6D13346924E05A876
:10DF800021464A4601960226009600F053FA002DDB
:10DF900006460DDA22684642636802F100422260BA
:10DFA00003F10043636003E00026002308604B6038
:10DFB000304609B0BDE8F08F0146002601F006FCAE
:10DFC00060602060F4E74FF488410126C3F23571A8
:10DFD00001F0FCFB4AF20831C2F68561054601F00A
:10DFE000F5FB01462060284601F0F0FB4AF20831BB
:10DFF000C2F6856101F0EAFB6060D9E700F0D0FE6F
:10E000004FF68411C3F62271074601F0E9FC4FF088
:10E010007C5101F0DDFB01F0A9FE064601F08CFC0D
:10E020004FF47861C3F6C971824601F0D9FC01460C
:10E03000384601F0CBFB44F24341C3F235718046D0
:10E04000504601F0CDFC1F2E8146404621DC4FF6A4
:10E05000FC73711EC0F601032BF0FF0253F8213050
:10E060009A4216D0494601F0B1FB07462060394676
:10E07000404601F0ABFB494601F0A8FB002D606073
:10E0800096DA07F1004700F10040276076426060B1
:10E090008EE749464FEAEB5B01F098FBC0F3C753AC
:10E0A0000746C3EB0B032060082BE0DD4FF48841EB
:10E0B0005046C3F2357101F093FC0746404639469D
:10E0C00001F084FB03904046039901F07FFB394641
:10E0D00001F07CFB4AF20831C2F6856107465046E2
:10E0E00001F07EFC394601F071FB814603984946F8
:10E0F00001F06CFBC0F3C7530746C3EB0B0B20606A
:10E10000BBF1190FD8BFDDF80C80B0DD4FF423410F
:10E110005046C2F6856101F063FC07460398394614
:10E1200001F054FB80460398414601F04FFB39460D
:10E1300001F04CFB43F23211C2F28D4107465046CA
:10E1400001F04EFC394601F041FB8146404689E72B
:10E1500001F03EFB4FF47D632BF00F0BC3F6C97348
:10E160009B45054614D044F243414FF0FF36C3F2BD
:10E17000357101F02DFB01462060284601F026FB99
:10E1800044F24341C3F2357101F022FB60600FE7B6
:10E190004FF488414FF0FF36C3F2357101F018FBA0
:10E1A0004AF20831C2F68561054601F011FB0146CD
:10E1B0002060284601F00AFB4AF20831C2F6856168
:10E1C00001F006FB6060F3E67C00020820F00042EC
:10E1D0000346B2F1FF4F70B5044639D2002A35D05C
:10E1E00000283FDBC115B2F5000F09D210F4000280
:10E1F00040D15B0001321802FBD5C2F1010289183F
:10E2000023F07F43A1F17F0223F40003D10743F4FD
:10E21000000348BF5B000026541019215B003546FF
:10E220004FF08072A8189842DEBFC0EB0303851838
:10E23000B61852085B000139F4D113B106F001039E
:10E240009E197610E40506F17C56A419204670BD8F
:10E25000014601F0C5FB0146204601F0B9FA04462B
:10E26000204670BD014601F0B1FA014601F06CFC98
:10E270000446EBE701228918C2E700BF2DE9F84305
:10E2800020F00046B6F1485F05460F465BDA01F024
:10E290006DFD002800F0CA802946284601F0A0FB49
:10E2A0004DF24E71CAF64751044601F099FB47F210
:10E2B000F641C3F20F1101F08BFA214601F090FBF9
:10E2C0004FF27C21C3F2934101F080FA214601F024
:10E2D00087FB40F60151C3F2D07101F079FA214673
:10E2E00001F07EFB40F66131C3F6B62101F06EFA13
:10E2F000214601F075FB4AF6AB21C3F62A5101F025
:10E3000067FA214601F06CFB804620464FF07C51B5
:10E3100001F066FB41460646204601F061FB3946A6
:10E320000446284601F05CFB0146204601F04EFA07
:10E330000146304601F04AFA01464FF07E5001F0A6
:10E3400045FABDE8F883014601F04AFB4DF24E71F3
:10E35000CAF64751044601F043FB47F2F641C3F2C7
:10E360000F1101F035FA214601F03AFB4FF27C2102
:10E37000C3F2934101F02AFA214601F031FB40F645
:10E380000151C3F2D07101F023FA214601F028FBBC
:10E3900040F66131C3F6B62101F018FA214601F0CA
:10E3A0001FFB4AF6AB21C3F62A5101F011FA2146B0
:10E3B00001F016FB49F69913C3F699639E42804615
:10E3C000A3DD0023C3F648739E4227DC06F17F4697
:10E3D0004FF07E50314601F0F9F9814620464FF06A
:10E3E0007C5101F0FDFA314601F0F0F94146064654
:10E3F000204601F0F5FA39460446284601F0F0FAC5
:10E400000146204601F0E2F90146304601F0DEF90E
:10E410000146484601F0DAF9BDE8F8834FF00009FB
:10E420000026C3F63879C3F69066D7E74FF07E50E2
:10E43000BDE8F8832DE9F04F151DDDB0D41E58BF9F
:10E44000254640F294340493013B0293ED10669B01
:10E45000C0F6020425EAE5750746099554F82340FD
:10E46000EB43089102EBC303029A07941619069333
:10E4700015D40136AD1A679B00240DF18008B60053
:10E4800003EB85090020002D03DB59F8040001F09F
:10E4900053FA48F8040004340135B442F2D1079C21
:10E4A000002C25DB079A48ABDDF810A00DF58E791E
:10E4B00003EB820B4FEA8A08029C0025002C11DB3B
:10E4C00020A8002400EB8A0600253859043456F8A9
:10E4D000041D01F085FA0146284601F079F944450A
:10E4E0000546F2D149F8045FD9450AF1010AE3D1A2
:10E4F000079A0CABDDF81C80013A0093C2460A92E1
:10E5000003EB82040B944FEA8A025CACA318BAF1C5
:10E51000000F019253F8504C22DD0DF590790BAEAF
:10E5200009EB02054FF06E51204601F059FA01F057
:10E530001DFC01F001FA4FF08741804601F050FACE
:10E540000146204601F042F901F010FC414646F830
:10E55000040F55F8040D01F03BF94D450446E1D197
:10E560000699204600F0ACFC4FF07851044601F0CB
:10E5700037FA00F019FC4FF0824101F031FA014600
:10E58000204601F023F9044601F0F0FB064601F0B5
:10E59000D3F90146204601F019F9069A002A0546EA
:10E5A00040F306810AF1FF330CA8C2F10801C2F161
:10E5B000070450F8232052FA01F0361810FA01F13E
:10E5C000521A0CA942FA04FB41F82320BBF1000FB8
:10E5D00030DD01360024BAF1000F17DD019C0CABD1
:10E5E0001919002407E022B10124C2F5807243F812
:10E5F000042C8B420AD053F8042B002CF3D00124B6
:10E600008B42C2F1FF0243F8042CF4D1069A002A8F
:10E610000DDD012A00F0D580022A08D10AF1FF336E
:10E620000CA951F8232002F03F0241F82320BBF14E
:10E63000020F6ED02846002101F066FB002800F092
:10E640008180079A0AF1FF34A2420FDC019A0CA8DC
:10E650008318079A00EB8200002253F8041D8342BE
:10E6600042EA0102F9D1002A40F0C3800A9C0CA8BA
:10E6700050F82430002B40F0BA800B9A012352F856
:10E68000041D01330029FAD053440AF101099945C8
:10E6900003933BDC099C029AA244679C02EB0903AA
:10E6A00020AA04EB8A0B049C013B059202EB830A2F
:10E6B0004FEA8408019B48AAD21801925BF8040F24
:10E6C000002501F039F9029A002A4AF8040F14DBF8
:10E6D000049B0025059A002409EB030602EB86063D
:10E6E0003859043456F8041D01F07AF901462846D9
:10E6F00001F06EF844450546F2D1039C09F1010989
:10E70000019BA14543F8045F0193D7DDDDF80CA020
:10E71000F9E629464FF07E5001F058F80546002CE6
:10E7200088D006994FF07E5000F0CAFB014628467B
:10E7300001F04CF800210546284601F0E5FA0028D2
:10E740007FF47FAF0296D0460AF1FF34002851D102
:10E75000069B2846594200F0B3FB4FF08741044620
:10E7600001F0F0FA002800F071814FF06E51204660
:10E7700001F036F9069A0AF101080832069201F012
:10E78000F5FA01F0D9F84FF08741054601F028F974
:10E790000146204601F01AF80CAC01F0E7FA0CAB88
:10E7A00043F82A00284601F0E1FA44F8280034E052
:10E7B00011D10AF1FF330CAA52F823304FEA232B70
:10E7C00004E70AF1FF330CA850F8232002F07F027F
:10E7D00040F823202BE74FF07C514FF0000B01F065
:10E7E000B1FA00283FF426AF4FF0020BF1E6012307
:10E7F0004AE702960CA8069AA04650F82430083A38
:10E80000069253B900EB8403A04653F8041D08F1A7
:10E81000FF38083A0029F8D006924FF07E5006994A
:10E8200000F04EFBB8F1000F05464CDB08F1010289
:10E830000CAB48A8019296009C19861954F8040D57
:10E8400001F07AF8294601F0CBF84FF06E5146F806
:10E85000040D284601F0C4F8009A94420546EDD113
:10E8600048ABCDF80C8003EB8809DFF8F0A1DDF8A8
:10E870001C800027B8F1000FC0F2DA80002FC0F230
:10E88000D78000240026254601E0BD420EDC59F861
:10E89000041001355AF80400043401F0A1F80146CF
:10E8A000304600F095FFA8450646EEDA5CAC019ACA
:10E8B00004EB87030137BA42A9F1040943F8A06CBD
:10E8C000D8D1DDF80C80669C032C14D8DFE804F066
:10E8D000986868190020BBF1000F59D0089B00F11F
:10E8E0000040089C349A9860359B02F100422260F7
:10E8F00003F100436360029A02F007005DB0BDE8D7
:10E90000F08FB8F1000FC4BF34AD05EB8804E1DD32
:10E9100054F8049C54F804794846394600F058FFEE
:10E9200006464846314600F051FF0146384600F0A1
:10E930004FFFAC4226606060EAD1B8F1010FC9DD3B
:10E9400008F1FF3405EB840454F80499A76848469D
:10E95000394600F03DFF06464846314600F036FF96
:10E960000146384600F034FFAC426660A060EBD14F
:10E9700008F1010804F10805002004EB880454F8AC
:10E98000041D00F025FFAC42F9D1BBF1000FA5D169
:10E99000089B089C9860349B2360359B6360AAE7C2
:10E9A0000020B8F1000F0BDB08F1010434AD0020AA
:10E9B00005EB840454F8041D00F00AFFAC42F9D1C1
:10E9C00000F10043BBF1000F00D10346089C014653
:10E9D0003498236000F0FAFEB8F1000F08DD34AC83
:10E9E00004EB880854F8041F00F0F2FE4445F9D106
:10E9F000BBF1000F01D000F10040089A50607AE7A7
:10EA00000020B8F1000F0BDB08F1010434AD002049
:10EA100005EB840454F8041D00F0DAFEAC42F9D191
:10EA2000BBF1000F01D000F10040089A106062E7CE
:10EA30005CAC019A04EB870301370026BA42A9F1C6
:10EA4000040943F8A06C7FF415AF3AE7204601F0C3
:10EA50008DF90CA941F82A00DFE600BFA0030208E7
:10EA60002DE9F84320F00043B3F1485F04460D461A
:10EA7000904603DA01F07AF9002859D02146204661
:10EA800000F0AEFF2146064600F0AAFF4CF6D31177
:10EA9000C2F62E710746304600F0A2FF42F63471EE
:10EAA000C3F2D72100F092FE314600F099FF4EF6F6
:10EAB0001B71C3F2386100F08BFE314600F090FF0D
:10EAC00040F60151C3F6501100F080FE314600F0CF
:10EAD00087FF48F68901C3F6084100F079FE8146B8
:10EAE000B8F1000F27D028464FF07C5100F078FF96
:10EAF00049468046384600F073FF0146404600F024
:10EB000065FE314600F06CFF294600F05FFE4AF6D4
:10EB1000AB21C3F62A610546384600F061FF014685
:10EB2000284600F055FE0146204600F04FFE044600
:10EB30002046BDE8F8830146304600F051FF4AF612
:10EB4000AB21C3F62A6100F041FE394600F048FFD0
:10EB50000146204600F03CFE04462046BDE8F8830E
:10EB6000002070472DE9F04120F00045B5F1A14F9C
:10EB7000044606460EDBB5F1FF4F00F3A4800028E3
:10EB800040F6DB74C8BFC3F6C97440F3D980204691
:10EB9000BDE8F0814FF6FF73C3F6DF639D4200F3DB
:10EBA000A780B5F1445FC0F295804FF0FF37214652
:10EBB000204600F015FF0146804600F011FF46F6A2
:10EBC000D711C3F68541054600F00AFF4DF65921DD
:10EBD000C3F64B5100F0FCFD294600F001FF46F65C
:10EBE0003531C3F6885100F0F3FD294600F0F8FEF8
:10EBF00042F66E61C3F6BA5100F0EAFD294600F014
:10EC0000EFFE44F62511C3F6126100F0E1FD29463E
:10EC100000F0E6FE4AF6AB21C3F6AA6100F0D8FD8B
:10EC2000414600F0DDFE4AF22121CBF61551804627
:10EC3000284600F0D5FE4FF26B11C3F66E5100F07E
:10EC4000C5FD294600F0CCFE48F29571C3F69D51F2
:10EC500000F0BCFD294600F0C3FE48F63861C3F65B
:10EC6000E35100F0B3FD294600F0BAFE4CF6CD4169
:10EC7000C3F64C6100F0AAFD294600F0B1FE7B1CF2
:10EC8000014651D040F2CC35404600F0A1FDC0F61F
:10EC90000205214600F0A4FE05EB8703196900F088
:10ECA00095FD214600F092FD014655F8270000F041
:10ECB0008DFD002EB8BF00F10044FFF668AF04469A
:10ECC0002046BDE8F081014600F082FD0446204662
:10ECD000BDE8F0814FF2CA21C7F2491100F078FD7A
:10ECE0004FF07E5101F038F800283FF45EAF4EE758
:10ECF00000F056F84FF6FF73C3F697739D424FF638
:10ED0000FF7304461FDCC3F62F739D423DDC0146B2
:10ED1000002700F05DFD4FF07E5100F057FD4FF0F1
:10ED20008041054620461FE0404600F051FD214647
:10ED300000F056FE0146204600F048FD044626E756
:10ED4000CBF6C97423E7C4F21B039D4214DC4FF0D9
:10ED50007F51022700F03AFD4FF07F5105462046D3
:10ED600000F03EFE4FF07E5100F032FD0146284695
:10ED700000F0EAFE04461AE700202146CBF6807038
:10ED8000032700F0E1FE044611E74FF07E51012712
:10ED900000F01CFD4FF07E5105462046E4E700BF21
:10EDA00020F00040704700BF2DE9F04120F0004600
:10EDB00001460446F50D7F3D162D1ADC002D8046D8
:10EDC00020DB4FF6FF77C0F27F072F4107420DD0BF
:10EDD0004FF2CA21C7F2491100F0FAFC002100F0FD
:10EDE000BBFF10B3002C24DB28EA07010846BDE86E
:10EDF000F081B6F1FF4FF9D300F0EAFC0146084676
:10EE0000BDE8F0814FF2CA21C7F2491100F0E0FCE1
:10EE1000002100F0A1FF40B10021002CE6DACBF682
:10EE20008071002E08BF2146E0E721460846BDE874
:10EE3000F0814FF4000353FA05F504EB050828EAC6
:10EE40000701D3E7D0F1010338BF0023B0F1004F31
:10EE500008BF43F001030BB102207047A0F5000387
:10EE600000F1FF42B3F1FE4F2CBF00230123B2F1AA
:10EE7000FE4F38BF43F001030BB1042070474FF63B
:10EE8000FE73411EC0F27F0300F10042013A994235
:10EE90008CBF002101219A428CBF0B4641F0010337
:10EEA0000BB10320704710F5000F14BF002301239E
:10EEB000B0F1FF4F14BF184643F00100704700BF88
:10EEC00010B50C4630F000410346024627D0B1F1A0
:10EED000FF4F26D2B1F5000F29D3C90D0919FE291C
:10EEE000C8BF194633DC0029C4BF22F0FF4242EA02
:10EEF000C15314DC11F1160F37DA4CF250321946B7
:10EF0000944224DC44F26020C0F6A25000F03AF8AB
:10EF100044F26021C0F6A25100F062FD034618469B
:10EF200010BD014600F054FC0346184610BD4FF0DA
:10EF3000984100F055FD43F6B042CFF6FF7294427F
:10EF40000346E5DBC0F3C75102461939C6E74FF265
:10EF5000CA20C7F2491000F015F84FF2CA21C7F2D3
:10EF6000491100F03DFD0346D9E701F1190022F0F7
:10EF7000FF424FF04C5142EAC05000F031FD0346D1
:10EF8000CDE700BF01F0004120F00040084370478A
:10EF900081F0004102E000BF83F0004330B54FEA4A
:10EFA00041044FEA430594EA050F08BF90EA020FB7
:10EFB0001FBF54EA000C55EA020C7FEA645C7FEA4A
:10EFC000655C00F0E2804FEA5454D4EB5555B8BF6D
:10EFD0006D420CDD2C4480EA020281EA030382EADE
:10EFE000000083EA010180EA020281EA0303362D70
:10EFF00088BF30BD11F0004F4FEA01314FF4801C43
:10F000004CEA113102D0404261EB410113F0004F54
:10F010004FEA03334CEA133302D0524263EB43030B
:10F0200094EA050F00F0A780A4F10104D5F1200EA9
:10F030000DDB02FA0EFC22FA05F2801841F1000104
:10F0400003FA0EF2801843FA05F359410EE0A5F1D8
:10F0500020050EF1200E012A03FA0EFC28BF4CF009
:10F06000020C43FA05F3C01851EBE37101F00045BF
:10F0700007D54FF0000EDCF1000C7EEB00006EEBCC
:10F080000101B1F5801F1BD3B1F5001F0CD3490856
:10F090005FEA30004FEA3C0C04F101044FEA4452AD
:10F0A00012F5800F80F09A80BCF1004F08BF5FEA34
:10F0B000500C50F1000041EB045141EA050130BD14
:10F0C0005FEA4C0C404141EB010111F4801FA4F1B7
:10F0D0000104E9D191F0000F04BF01460020B1FA0C
:10F0E00081F308BF2033A3F10B03B3F120020CDA44
:10F0F0000C3208DD02F1140CC2F10C0201FA0CF022
:10F1000021FA02F10CE002F11402D8BFC2F1200C86
:10F1100001FA02F120FA0CFCDCBF41EA0C0190403C
:10F12000E41AA2BF01EB0451294330BD6FEA040485
:10F130001F3C1CDA0C340EDC04F11404C4F1200270
:10F1400020FA04F001FA02F340EA030021FA04F382
:10F1500045EA030130BDC4F10C04C4F1200220FAD9
:10F1600002F001FA04F340EA0300294630BD21FA17
:10F1700004F0294630BD94F0000F83F4801306BFDD
:10F1800081F480110134013D4EE77FEA645C18BFD1
:10F190007FEA655C29D094EA050F08BF90EA020F68
:10F1A00005D054EA000C04BF1946104630BD91EA60
:10F1B000030F1EBF0021002030BD5FEA545C05D163
:10F1C0004000494128BF41F0004130BD14F58004A2
:10F1D0003CBF01F5801130BD01F0004545F0FE4116
:10F1E00041F470014FF0000030BD7FEA645C1ABF4B
:10F1F000194610467FEA655C1CBF0B46024650EA82
:10F20000013406BF52EA033591EA030F41F40021AD
:10F2100030BD00BF90F0000F04BF0021704730B533
:10F220004FF4806404F132044FF000054FF0000108
:10F2300050E700BF90F0000F04BF0021704730B5C9
:10F240004FF4806404F1320410F0004548BF40429E
:10F250004FF000013EE700BF42004FEAE2014FEAF3
:10F2600031014FEA02701FBF12F07F4393F07F4FCE
:10F2700081F06051704792F0000F14BF93F07F4F00
:10F28000704730B54FF4607401F0004521F0004143
:10F2900020E700BF50EA010208BF704730B54FF0C9
:10F2A00000050AE050EA010208BF704730B511F0CE
:10F2B000004502D5404261EB41014FF4806404F106
:10F2C00032045FEA915C3FF4DCAE4FF003025FEA88
:10F2D000DC0C18BF03325FEADC0C18BF033202EB10
:10F2E000DC02C2F1200300FA03FC20FA02F001FA6A
:10F2F00003FE40EA0E0021FA02F11444C1E600BF09
:10F3000070B54FF0FF0C4CF4E06C1CEA11541DBFBB
:10F310001CEA135594EA0C0F95EA0C0F00F0DEF886
:10F320002C4481EA030621EA4C5123EA4C5350EA6B
:10F33000013518BF52EA033541F4801143F48013BC
:10F3400038D0A0FB02CE4FF00005E1FB02E506F04D
:10F350000042E0FB03E54FF00006E1FB03569CF0A2
:10F36000000F18BF4EF0010EA4F1FF04B6F5007FA8
:10F3700064F5407404D25FEA4E0E6D4146EB06061A
:10F3800042EAC62141EA55514FEAC52040EA5E50A3
:10F390004FEACE2EB4F1FD0C88BFBCF5E06F1ED84D
:10F3A000BEF1004F08BF5FEA500E50F1000041EB84
:10F3B000045170BD06F0004646EA010140EA020031
:10F3C00081EA0301B4EB5C04C2BFD4EB0C0541EA53
:10F3D000045170BD41F480114FF0000E013C00F368
:10F3E000AB8014F1360FDEBF002001F0004170BD8C
:10F3F000C4F10004203C35DA0C341BDC04F11404A5
:10F40000C4F1200500FA05F320FA04F001FA05F230
:10F4100040EA020001F0004221F0004110EBD370FD
:10F4200021FA04F642EB06015EEA430E08BF20EA29
:10F43000D37070BDC4F10C04C4F1200500FA04F3CC
:10F4400020FA05F001FA04F240EA020001F000415E
:10F4500010EBD37041F100015EEA430E08BF20EAD1
:10F46000D37070BDC4F1200500FA05F24EEA020E19
:10F4700020FA04F301FA05F243EA020321FA04F048
:10F4800001F0004121FA04F220EA020000EBD370FF
:10F490005EEA430E08BF20EAD37070BD94F0000FFF
:10F4A0000FD101F00046400041EB010111F4801F33
:10F4B00008BF013CF7D041EA060195F0000F18BFE4
:10F4C000704703F00046520043EB030313F4801F20
:10F4D00008BF013DF7D043EA0603704794EA0C0FDA
:10F4E0000CEA135518BF95EA0C0F0CD050EA4106F0
:10F4F00018BF52EA4306D1D181EA030101F000416D
:10F500004FF0000070BD50EA410606BF1046194694
:10F5100052EA430619D094EA0C0F02D150EA0136A0
:10F5200013D195EA0C0F05D152EA03361CBF1046E1
:10F5300019460AD181EA030101F0004141F0FE4180
:10F5400041F470014FF0000070BD41F0FE4141F404
:10F55000780170BD70B54FF0FF0C4CF4E06C1CEA04
:10F5600011541DBF1CEA135594EA0C0F95EA0C0FB9
:10F5700000F0A7F8A4EB050481EA030E52EA033574
:10F580004FEA013100F088804FEA03334FF0805595
:10F5900045EA131343EA12634FEA022245EA1115C2
:10F5A00045EA10654FEA00260EF000419D4208BF73
:10F5B000964244F1FD0404F5407402D25B084FEA20
:10F5C0003202B61A65EB03055B084FEA32024FF4CC
:10F5D00080104FF4002CB6EB020E75EB030E22BF29
:10F5E000B61A754640EA0C005B084FEA3202B6EBE9
:10F5F000020E75EB030E22BFB61A754640EA5C0098
:10F600005B084FEA3202B6EB020E75EB030E22BF27
:10F61000B61A754640EA9C005B084FEA3202B6EB28
:10F62000020E75EB030E22BFB61A754640EADC00E7
:10F6300055EA060E18D04FEA051545EA16754FEA49
:10F6400006164FEAC30343EA52734FEAC2025FEA67
:10F650001C1CC0D111F4801F0BD141EA00014FF0F6
:10F6600000004FF0004CB6E711F4801F04BF0143C7
:10F670000020B4F1FD0C88BFBCF5E06F3FF6AFAEE3
:10F68000B5EB030C04BFB6EB020C5FEA500C50F173
:10F69000000041EB045170BD0EF0004E4EEA1131F6
:10F6A00014EB5C04C2BFD4EB0C0541EA045170BDFD
:10F6B00041F480114FF0000E013C90E645EA060E41
:10F6C0008DE60CEA135594EA0C0F08BF95EA0C0F6F
:10F6D0003FF43BAF94EA0C0F0AD150EA01347FF4B7
:10F6E00034AF95EA0C0F7FF425AF104619462CE78E
:10F6F00095EA0C0F06D152EA03353FF4FDAE1046F1
:10F70000194622E750EA410618BF52EA43067FF441
:10F71000C5AE50EA41047FF40DAF52EA43057FF4D1
:10F72000EBAE12E74FEA4102B2F1E04324BFB3F57A
:10F73000001CDCF1FE5C0DD901F0004C4FEAC00268
:10F740004CEA5070B2F1004F40EB830008BF20F04C
:10F750000100704711F0804F21D113F13872BCBF06
:10F7600001F00040704741F480114FEA5252C2F15B
:10F770001802C2F1200C10FA0CF320FA02F018BFA4
:10F7800040F001004FEAC1234FEAD32303FA0CFCF7
:10F7900040EA0C0023FA02F34FEA4303CCE77FEA86
:10F7A000625307D150EA01331EBF4FF0FE4040F4D0
:10F7B0004000704701F0004040F0FE4040F400007F
:10F7C000704700BF80F0004002E000BF81F00041C0
:10F7D00042001FBF5FEA410392EA030F7FEA226CF7
:10F7E0007FEA236C6AD04FEA1262D2EB1363C1BF87
:10F7F000D218414048404140B8BF5B42192B88BFF6
:10F80000704710F0004F40F4000020F07F4018BF18
:10F81000404211F0004F41F4000121F07F4118BF38
:10F82000494292EA030F3FD0A2F1010241FA03FCE0
:10F8300010EB0C00C3F1200301FA03F100F00043C8
:10F8400002D5494260EB4000B0F5000F13D3B0F190
:10F85000807F06D340084FEA310102F10102FE2AFF
:10F8600051D2B1F1004F40EBC25008BF20F001006F
:10F8700040EA03007047490040EB000010F4000F1D
:10F88000A2F10102EDD1B0FA80FCACF1080CB2EBB0
:10F890000C0200FA0CF0AABF00EBC250524218430F
:10F8A000BCBFD0401843704792F0000F81F40001B4
:10F8B00006BF80F400000132013BB5E74FEA410387
:10F8C0007FEA226C18BF7FEA236C21D092EA030FF3
:10F8D00004D092F0000F08BF0846704790EA010F6D
:10F8E0001CBF0020704712F07F4F04D1400028BF9A
:10F8F00040F00040704712F100723CBF00F500007C
:10F90000704700F0004343F0FE4040F400007047B1
:10F910007FEA226216BF08467FEA2363014642025D
:10F9200006BF5FEA412390EA010F40F48000704770
:10F930004FF0000304E000BF10F0004348BF404216
:10F940005FEA000C08BF704743F0964301464FF052
:10F9500000001CE050EA010208BF70474FF00003AE
:10F960000AE000BF50EA010208BF704711F00043EF
:10F9700002D5404261EB41015FEA010C02BF8446BF
:10F980000146002043F0B64308BFA3F18053A3F51E
:10F990000003BCFA8CF2083AA3EBC25310DB01FA65
:10F9A00002FC634400FA02FCC2F12002BCF1004FE9
:10F9B00020FA02F243EB020008BF20F0010070477A
:10F9C00002F1200201FA02FCC2F1200250EA4C00CE
:10F9D00021FA02F243EB020008BF20EADC70704714
:10F9E0004FF0FF0C1CEAD0521EBF1CEAD15392EA22
:10F9F0000C0F93EA0C0F6FD01A4480EA010C4002FE
:10FA000018BF5FEA41211ED04FF0006343EA501057
:10FA100043EA5111A0FB01310CF00040B1F5000F99
:10FA20003EBF490041EAD3715B0040EA010062F148
:10FA30007F02FD2A1DD8B3F1004F40EBC25008BF32
:10FA400020F00100704790F0000F0CF0004C08BF50
:10FA500049024CEA502040EA51207F3AC2BFD2F11D
:10FA6000FF0340EAC250704740F400004FF000032B
:10FA7000013A5DDC12F1190FDCBF00F00040704765
:10FA8000C2F10002410021FA02F1C2F1200200FAA3
:10FA900002FC5FEA310040F1000053EA4C0308BF6A
:10FAA00020EADC70704792F0000F00F0004C02BFBB
:10FAB000400010F4000F013AF9D040EA0C0093F036
:10FAC000000F01F0004C02BF490011F4000F013B90
:10FAD000F9D041EA0C018FE70CEAD15392EA0C0FFE
:10FAE00018BF93EA0C0F0AD030F0004C18BF31F069
:10FAF000004CD8D180EA010000F00040704790F03F
:10FB0000000F17BF90F0004F084691F0000F91F0E2
:10FB1000004F14D092EA0C0F01D142020FD193EAA8
:10FB20000C0F03D14B0218BF084608D180EA010030
:10FB300000F0004040F0FE4040F40000704740F00C
:10FB4000FE4040F4400070474FF0FF0C1CEAD052DA
:10FB50001EBF1CEAD15392EA0C0F93EA0C0F69D036
:10FB6000A2EB030280EA010C49024FEA402037D0A1
:10FB70004FF0805343EA111143EA10130CF0004098
:10FB80008B4238BF5B0042F17D024FF4000C8B4288
:10FB900024BF5B1A40EA0C00B3EB510F24BFA3EB68
:10FBA000510340EA5C00B3EB910F24BFA3EB910338
:10FBB00040EA9C00B3EBD10F24BFA3EBD10340EA92
:10FBC000DC001B0118BF5FEA1C1CE0D1FD2A3FF6D8
:10FBD00050AF8B4240EBC25008BF20F0010070478D
:10FBE0000CF0004C4CEA50207F32C2BFD2F1FF0330
:10FBF00040EAC250704740F400004FF00003013A61
:10FC000037E792F0000F00F0004C02BF400010F404
:10FC1000000F013AF9D040EA0C0093F0000F01F018
:10FC2000004C02BF490011F4000F013BF9D041EA3A
:10FC30000C0195E70CEAD15392EA0C0F08D142026D
:10FC40007FF47DAF93EA0C0F7FF470AF084676E740
:10FC500093EA0C0F04D14B023FF44CAF08466EE719
:10FC600030F0004C18BF31F0004CCAD130F00042E7
:10FC70007FF45CAF31F000437FF43CAF5FE700BF3F
:10FC80004FF0FF3C06E000BF4FF0010C02E000BF68
:10FC90004FF0010C4DF804CD4FEA40024FEA41030A
:10FCA0007FEA226C18BF7FEA236C11D001B052EAC0
:10FCB000530C18BF90EA010F58BFB2EB030088BF86
:10FCC000C81738BF6FEAE17018BF40F001007047F5
:10FCD0007FEA226C02D15FEA402C05D17FEA236CD7
:10FCE000E4D15FEA412CE1D05DF8040B704700BF1E
:10FCF000844608466146FFE70FB5FFF7C9FF0028B5
:10FD000048BF10F1000F0FBD4DF808EDFFF7F4FFED
:10FD10000CBF012000205DF808FB00BF4DF808ED86
:10FD2000FFF7EAFF34BF012000205DF808FB00BFA9
:10FD30004DF808EDFFF7E0FF94BF012000205DF8CB
:10FD400008FB00BF4DF808EDFFF7D2FF94BF01207C
:10FD500000205DF808FB00BF4DF808EDFFF7C8FF75
:10FD600034BF012000205DF808FB00BF4FEA4002CD
:10FD7000B2F1FE4F0FD34FF09E03B3EB12620DD9D9
:10FD80004FEA002343F0004310F0004F23FA02F043
:10FD900018BF404270474FF00000704712F1610FEA
:10FDA00001D1420205D110F0004008BF6FF00040C1
:10FDB00070474FF00000704742000ED2B2F1FE4F84
:10FDC0000BD34FF09E03B3EB126209D44FEA00232A
:10FDD00043F0004323FA02F070474FF000007047F1
:10FDE00012F1610F01D1420202D14FF0FF30704792
:10FDF0004FF00000704700BF43F21003C2F200034F
:10FE00001868704720F0030110F00300C0F10000F3
:10FE100051F8043B00F1040C4FEACC0C6FF00002E7
:10FE20001CBF22FA0CF213434FF0010C4CEA0C2CCD
:10FE30004CEA0C4CA3EB0C0222EA030212EACC12AD
:10FE400004BF51F8043B0430F4D013F0FF0F1FBF80
:10FE5000013013F47F4F013013F47F0F18BF0130CE
:10FE6000704700BF536176696E6720524F4D20691D
:10FE70006D6167652C202538642062797465732074
:10FE80006C656674202020200000000053617669B4
:10FE90006E6720524F4D20696D6167652E2E2E00D2
:10FEA000666C6173682E62696E000000666C617337
:10FEB000682E62696E207361766564202D20636808
:10FEC00065636B73756D2069732025642020202085
:10FED00020000000424DF6BB00000000000076004C
:10FEE00000002800000090010000F0000000010068
:10FEF00004000000000080BB0000701700007017B5
:10FF00000000100000000000000000002020202061
:10FF100020202020202020202020202020202020E1
:10FF200020202020202020202020202020202020D1
:10FF300020202020202020202020202020202020C1
:10FF400020202020202020202020202020202020B1
:10FF500020202000202020202020202020202020C1
:10FF60002020202020202020484152444641554C4A
:10FF7000542020202020202020202020202020204D
:10FF8000200000000A53503A200000002020504377
:10FF90003A20000020204C523A2000000A524547E7
:10FFA000533A2072302000002C20723120000000D3
:10FFB0000A20202020202072322000002C207233C2
:10FFC000200000002C207231322000000A534342EE
:10FFD00020484653523A20000A5343422043465396
:10FFE000523A20000A535441434B2044554D503A55
:10FFF0000A0000007371727466000000000FC93FB0
:020000040802F0
:10000000000F494000CB9640000FC9400053FB4011
:1000100000CB164100ED2F41000F494100316241F4
:1000200000537B41003A8A4100CB9641005CA341DA
:1000300000EDAF41007EBC41000FC94100A0D54199
:100040000031E24100C2EE410053FB4100F20342A5
:10005000003A0A420083104200CB164200141D42AF
:10006000005C234200A5294200ED2F4200363642B3
:10007000007E3C4200C74242000F4942A2000000FD
:10008000F9000000830000006E0000004E00000038
:10009000440000001500000029000000FC000000E2
:1000A0002700000057000000D1000000F50000000C
:1000B00034000000DD000000C0000000DB00000094
:1000C0006200000095000000990000003C00000064
:1000D000430000009000000041000000FE0000000E
:1000E0005100000063000000AB000000DE000000D3
:1000F000BB000000C500000061000000B700000068
:10010000240000006E0000003A00000042000000E1
:100110004D000000D2000000E000000006000000DA
:10012000490000002E000000EA0000000900000065
:10013000D1000000920000001C000000FE00000042
:100140001D000000EB0000001C000000B1000000DA
:1001500029000000A70000003E000000E8000000A9
:100160008200000035000000F50000002E000000B5
:10017000BB0000004400000084000000E900000013
:100180009C0000007000000026000000B400000089
:100190005F0000007E000000410000003900000008
:1001A00091000000D600000039000000830000002C
:1001B0005300000039000000F40000009C00000023
:1001C000840000005F0000008B000000BD00000004
:1001D000F9000000280000003B0000001F000000A4
:1001E000F800000097000000FF000000DE000000A3
:1001F00005000000980000000F000000EF00000064
:100200002F000000110000008B0000005A000000C9
:100210000A0000006D0000001F0000006D000000DB
:10022000360000007E000000CF0000002700000024
:10023000CB00000009000000B70000004F000000E4
:10024000460000003F000000660000009E00000025
:100250005F000000EA0000002D00000075000000B3
:1002600027000000BA000000C7000000EB000000FB
:10027000E5000000F10000007B0000003D000000F0
:100280000700000039000000F70000008A000000AD
:100290005200000092000000EA0000006B00000025
:1002A000FB0000005F000000B10000001F00000024
:1002B0008D0000005D0000000800000056000000F6
:1002C000030000003000000046000000FC000000B9
:1002D0007B0000006B000000AB000000F00000009D
:1002E000CF000000BC000000200000009A000000C9
:1002F000F4000000360000001D000000A90000000E
:10030000E300000091000000610000005E000000BA
:10031000E60000001B00000008000000650000006F
:1003200099000000850000005F000000140000003C
:10033000A000000068000000400000008D000000E8
:10034000FF000000D8000000800000004D00000009
:1003500073000000270000003100000006000000CC
:10036000060000001500000056000000CA00000052
:1003700073000000A8000000C90000006000000039
:10038000E20000007B000000C00000008C000000C4
:100390006B000000040000000700000009000000DE
:1003A0000000C93F0000F0390000DA370000A23336
:1003B0000000842E0000502B0000C2270000D02235
:1003C0000000C41F0000C61B000044173863ED3E48
:1003D000DA0F493F5E987B3FDA0FC93F6937AC318E
:1003E00068212233B40F14336821A2331430002063
:0403F00043000000C6
:1003F40004000000DC0000001F00140001000000E5
:100404001430002000000000000000000000000084
:1004140000000000000000000000000000000000D8
:1004240000000000F00302080000000000000000CB
:1004340000000000000000000000000000000000B8
:1004440000000000000000000000000000000000A8
:100454000000000000000000000000000000000098
:100464000000000000000000000000000000000088
:100474000000000000000000000000000000000078
:100484000000000000000000000000000000000068
:100494000000000000000000000000000000000058
:1004A4000000000000000000000000000000000048
:1004B4000000000000000000000000000000000038
:1004C4000000000000000000000000000000000028
:1004D4000000000000000000000000000000000018
:1004E4000000000000000000000000000000000008
:0404F4000000000004
:040000050801D78592
:00000001FF
